:100000000C9485000C94AD000C94AD000C94AD00E4
:100010000C94AD000C94AD000C94AD000C94AD00AC
:100020000C94AD000C94AD000C94AD000C94AD009C
:100030000C94AD000C94AD000C94AD000C94AD008C
:100040000C942E030C94AD000C9469020C944302A2
:100050000C94AD000C94AD000C94AD000C94AD006C
:100060000C94AD000C94AD00B4061707E106C90668
:100070001D081D08AE061D08AE061D08AE06AE061C
:10008000AE061D08AE06AE06FF0A660B910BE40B2A
:10009000530CA40CEE0CB70CC10CCA0CEE0CEE0CFD
:1000A000EE0CEE0C1D0B4B0B0C0CB70B490C0000AF
:1000B0000000240027002A0000000000250028007E
:1000C0002B00000000002300260029000404040483
:1000D00004040404020202020202030303030303F2
:1000E00001020408102040800102040810200102CF
:1000F00004081020000000080002010000030407AB
:1001000000000000000000001A1211241FBECFEFF3
:10011000D8E0DEBFCDBF11E0A0E0B1E0EEE9F7E24C
:1001200002C005900D92AC35B107D9F725E0ACE5DA
:10013000B1E001C01D92A432B207E1F710E0C5E8BA
:10014000D0E004C02197FE010E947F13C438D1077C
:10015000C9F70E94020D0C94CD130C940000CF92AD
:10016000DF92EF92FF920F931F93CF93DF936C0177
:100170007A018B01C0E0D0E0CE15DF0589F0D8010F
:100180006D918D01D601ED91FC910190F081E02DF2
:10019000C6010995892B11F47E0102C02196ECCF8E
:1001A000C701DF91CF911F910F91FF90EF90DF90EA
:1001B000CF900895089580E090E00895FC01538D5C
:1001C000448D252F30E0842F90E0821B930B541731
:1001D00010F0CF96089501970895FC01918D828DBE
:1001E000981761F0828DDF01A80FB11D5D968C918B
:1001F000928D9F5F9F73928F90E008958FEF9FEF96
:100200000895FC01918D828D981731F0828DE80F51
:10021000F11D858D90E008958FEF9FEF0895FC010B
:10022000918D228D892F90E0805C9F4F821B9109D8
:100230008F739927089587E193E00E940F0121E0D1
:10024000892B09F420E0822F0895FC01848DDF01C1
:10025000A80FB11DA35ABF4F2C91848D90E0019639
:100260008F739927848FA689B7892C93A089B18928
:100270008C9180648C93938D848D981306C0028832
:10028000F389E02D80818F7D80830895EF92FF9226
:100290000F931F93CF93DF93EC0181E0888F9B8DA9
:1002A0008C8D981305C0E889F989808185FD24C06B
:1002B000F62E0B8D10E00F5F1F4F0F731127E02EEE
:1002C0008C8DE8120CC00FB607FCFACFE889F989CB
:1002D000808185FFF5CFCE010E942501F1CF8B8D66
:1002E000FE01E80FF11DE35AFF4FF0820B8FEA8900
:1002F000FB898081806207C0EE89FF896083E8897D
:10030000F98980818064808381E090E0DF91CF91E2
:100310001F910F91FF90EF900895CF93DF93EC0121
:10032000888D8823C9F0EA89FB89808185FD05C015
:10033000A889B9898C9186FD0FC00FB607FCF5CF4F
:10034000808185FFF2CFA889B9898C9185FFEDCF97
:10035000CE010E942501E7CFDF91CF91089580E083
:1003600090E0892B29F00E941B0181110C94000060
:100370000895CF93DF9390E0FC01E052FF4F24916A
:10038000FC01E453FF4F8491882361F190E0880FD2
:10039000991FFC01E255FF4FC591D491FC01E8542F
:1003A000FF4FA591B491611109C09FB7F89488815E
:1003B000209582238883EC912E230BC0623061F458
:1003C0009FB7F8943881822F809583238883EC919E
:1003D0002E2B2C939FBF06C08FB7F894E8812E2B4D
:1003E00028838FBFDF91CF9108953FB7F894809114
:1003F000510290915202A0915302B091540226B53D
:10040000A89B05C02F3F19F00196A11DB11D3FBF4C
:10041000BA2FA92F982F8827820F911DA11DB11DDA
:10042000BC01CD0142E0660F771F881F991F4A95D6
:10043000D1F708952FB7F89460914D0270914E0254
:1004400080914F02909150022FBF08950E94C813CF
:100450006D3F71053CF46A3F710554F4683F7105C6
:1004600089F406C09B012E5F31092230310550F41A
:10047000DC018D919C91DC01ED91FC910190F0816A
:10048000E02D099408951F920F920FB60F92112438
:100490002F933F934F935F936F937F938F939F938C
:1004A000AF93BF93EF93FF9387E193E00E94250101
:1004B000FF91EF91BF91AF919F918F917F916F913C
:1004C0005F914F913F912F910F900FBE0F901F9012
:1004D00018951F920F920FB60F9211242F938F939E
:1004E0009F93EF93FF93E0912703F091280380817E
:1004F000E0912D03F0912E0382FD12C09081809136
:1005000030038F5F8F7320913103821751F0E09198
:100510003003F0E0E95EFC4F958F8093300301C01B
:100520008081FF91EF919F918F912F910F900FBE3E
:100530000F901F901895833081F028F4813099F046
:100540008230A1F008958730A9F08830B9F0843066
:10055000D1F4809180008F7D03C0809180008F77DF
:1005600080938000089584B58F7702C084B58F7D15
:1005700084BD08958091B0008F7703C08091B00052
:100580008F7D8093B00008951F93CF93DF93282F22
:1005900030E0F901EC50FF4F8491F901E052FF4F38
:1005A000D491F901E453FF4FC491CC23C9F0162F25
:1005B00081110E949B02EC2FF0E0EE0FFF1FE85428
:1005C000FF4FA591B4918FB7F894111105C09C917C
:1005D000ED2FE095E92302C0EC91ED2BEC938FBF5A
:1005E000DF91CF911F9108958F929F92AF92BF920A
:1005F000CF92DF92EF92FF926B017C010E94F50196
:100600004B015C01C114D104E104F104F1F00E943A
:10061000F501DC01CB0188199909AA09BB09883EBB
:100620009340A105B10570F321E0C21AD108E10899
:10063000F10888EE880E83E0981EA11CB11CC1143D
:10064000D104E104F10419F7DDCFFF90EF90DF90C2
:10065000CF90BF90AF909F908F9008951F920F9270
:100660000FB60F9211242F933F938F939F93AF93C5
:10067000BF9380914D0290914E02A0914F02B09194
:10068000500230914C0223E0230F2D3720F40196C5
:10069000A11DB11D05C026E8230F0296A11DB11DA5
:1006A00020934C0280934D0290934E02A0934F02F0
:1006B000B09350028091510290915202A091530246
:1006C000B09154020196A11DB11D809351029093E7
:1006D0005202A0935302B0935402BF91AF919F91E5
:1006E0008F913F912F910F900FBE0F901F901895F3
:1006F000AF92BF92CF92DF92EF92FF921F93CF9370
:10070000DF9300D0CDB7DEB77C016B0191E0122FF3
:10071000192759F060EF70E0D7018D919C914983C2
:100720005A830E94FB0C5A8149815A01C40ED51E7E
:10073000AC14BD0471F0F70180819181D5016D91F8
:100740005D01DC01ED91FC910190F081E02D0995B6
:10075000EFCF112391F067EF70E0F7018081918175
:100760000F900F90DF91CF911F91FF90EF90DF904E
:10077000CF90BF90AF900C94FB0C0F900F90DF9137
:10078000CF911F91FF90EF90DF90CF90BF90AF90EF
:1007900008950F931F93CF93DF931F92CDB7DEB7CA
:1007A0008C0169830E9406136981681741F0C801B2
:1007B0000F90DF91CF911F910F910C940E130F901A
:1007C000DF91CF911F910F9108950C94061387FF2D
:1007D0000DC09CE0980F923048F0982F9B7F993F76
:1007E00029F0803F08F4807F90E0089580E090E059
:1007F0000895EF92FF921F93CF93DF931F92CDB78F
:10080000DEB77C01162F2150203108F04EC080E861
:10081000E816F1040CF449C0A1EEEA16F104ACF5B7
:100820008091D8039091D903DC01ED91FC916E2D5C
:10083000622B0190F081E02D498309958091D803C6
:100840009091D903DC01ED91FC91612F6F770190BC
:10085000F081E02D0995E894E4F84981B0ECEB16BD
:10086000F10419F18091D8039091D903DC01ED9145
:10087000FC91642F6F770190F081E02D0F90DF9154
:10088000CF911F91FF90EF900994C701885F910964
:10089000089758F4B70188ED93E00F90DF91CF915E
:1008A0001F91FF90EF900C9428020F90DF91CF9151
:1008B0001F91FF90EF9008950F93082FEEE0F3E063
:1008C00021E030E040E050E060E070E080E090E067
:1008D0000E948513209530954095509560957095B0
:1008E00080959095A0812A23208321813223318312
:1008F0002281422342832381522353832481622312
:100900006483258172237583268182238683878170
:10091000982397830F910895242F462F682F80EBFB
:1009200090E00C94F903EF92FF920F931F93CF93F3
:10093000DF93D091DA03D13108F09DC28091D803C2
:100940009091D903DC01ED91FC910084F185E02DBB
:100950000995892B09F48FC28091D8039091D9030E
:10096000DC01ED91FC910284F385E02D09958C0169
:100970008B7F893F09F47FC22091E2033091E3032A
:100980002115310509F0AFC00093DD03C091DB03F1
:100990008C2F0E94E7030E947308882361F007FDF3
:1009A0000AC0C093DD030093DE0381E090E09093E2
:1009B000E3038093E203C091DD038C2F0E94E703E1
:1009C000813F910509F461C084F5803B910509F4EC
:1009D0005FC06CF48039910509F45AC0803A9105E2
:1009E00009F456C08038910509F0DBC051C0803D44
:1009F000910509F44AC02CF4803C910509F445C0E6
:100A0000D0C0803E910509F443C0803F910509F0B4
:100A1000C8C020E830E03093E1032093E003109257
:100A2000DB0320EF2093EE0339C0883F9105B9F036
:100A300044F4833F910549F15CF1863F910579F0DB
:100A4000B0C08A3F91050CF4ACC08D3F91053CF0DD
:100A50009C012E5F31092230310508F0A2C090932D
:100A6000EB038093EA031092E9031092EC031092D7
:100A7000ED0381E080936E041092E3031092E20391
:100A80001092E1031092E003EAC022E030E002C0DD
:100A900023E030E03093E1032093E0032091E20370
:100AA0003091E3034091E0035091E103415051093B
:100AB0002417350708F4CCC09093EB038093EA0326
:100AC000CF70CF5FC093E9038091DE038093EC0386
:100AD0001092ED031092E3031092E2031092E103EF
:100AE0001092E00321C007FF46C0C80199278D3F3F
:100AF000910554F48A3F91056CF4873F9105C1F04C
:100B0000883F9105C1F506C0AC014E5F51094230E6
:100B1000510588F59093EB038093EA031092EC0360
:100B20001092ED031092E90381E080936E0497C068
:100B30008091EE03803FA9F5C9010196F901EC54BB
:100B4000FC4F47EF42AF20EF30E03093EB032093B0
:100B5000EA038093EC039093ED031092E90381E0A4
:100B600080936E041092E3031092E2031092E1036B
:100B70001092E0036AC08091DD03F901EC54FC4F50
:100B8000803FD1F402AFE090E003F090E103C701B1
:100B900001972817390708F45BC0C091DD03C03FF7
:100BA00069F41092E3031092E2031092E1031092B1
:100BB000E0031092DB035FC101A7E5CF8C2F0E94F9
:100BC000E7038C019093EB038093EA030E94730880
:100BD000882331F08C2F8F708F5F8093E90302C0E0
:100BE0001092E9038091DE038093EC03B3E0EB16EF
:100BF000F10419F48091DF0301C080E08093ED03DC
:100C00001092E3031092E2031092E1031092E003CA
:100C100081E080936E04003B1105A1F054F400398B
:100C2000110581F0003A110569F00038110569F4E9
:100C300009C0003D110531F0003E110519F0003CDE
:100C4000110519F4C093DB030AC01092DB0307C03F
:100C50002F5F3F4F3093E3032093E2030CC1809159
:100C6000EA039091EB038039910529F48091ED031B
:100C7000882309F402C18091EA039091EB039C015F
:100C8000205831092136310508F0FEC02091E903D2
:100C90002D1709F4F9C0DD2309F4F6C0C0E01EC029
:100CA000813D91050CF446C1803E910509F053C188
:100CB000E091C003F091C103309779F06091ED03AA
:100CC0006F7720E8629FB00111248091EC038F7749
:100CD000682B70528091E9030995C1E04091E803C7
:100CE000342F317040FFA9C1842F8E7F09F4A5C134
:100CF0008091EA039091EB03BC0160587109613661
:100D0000710508F52091E9032D1719F031E0D11193
:100D100030E0469550E04230510541F043305105F6
:100D200049F04130510509F088C106C0332309F468
:100D300084C102C0311181C14091ED036091EC0387
:100D40000E94F9037AC1FC01E05FF109E031F1058D
:100D500008F073C1EC5CFF4F0C947F13BC0188ED6D
:100D600093E00E94280269C16091ED0370E0762F44
:100D700066278091EC03682B6138710510F060E8FC
:100D800070E021E04EEE53E088ED93E00E9478039E
:100D900054C1D091EC038091D8039091D903DC0128
:100DA000ED91FC910190F081E02D63EF0995DF77E3
:100DB0006D2F70E08091D8039091D9030E94FB0CB5
:100DC0003CC10091ED03B0E80B9F8001112480919C
:100DD000EC03082B8091D8039091D903DC01ED91AD
:100DE000FC910190F081E02D62EF09958091D8038C
:100DF0009091D903DC01ED91FC91B8016F777727D1
:100E00000190F081E02D09958091D8039091D9034C
:100E1000DC01ED91FC91B801660F672F661F770B1F
:100E200071956F7777270190F081E02D22C0809136
:100E3000EC038770B0E18B9FC0011124D091ED03CA
:100E4000DF70D82B8091D8039091D903DC01ED910C
:100E5000FC910190F081E02D61EF09958091D8031C
:100E60009091D903DC01ED91FC910190F081E02D8E
:100E70006D2F0995E2C0C0E0E0C080E890E090935B
:100E8000EB038093EA03F7CE813F9105C1F4E09133
:100E9000C403F091C5030CC08B3F91050CF0ACC0AE
:100EA000833F910509F089C0E091C803F091C9031F
:100EB000309709F412CF8091EC0309950ECF823F51
:100EC00091050CF064C0803B9105C1F4E091BA0338
:100ED000F091BB0308C08038910509F0FECEE09187
:100EE000B403F091B503309709F4F7CE4091ED03C8
:100EF0006091EC038091E9030995EFCE813B910568
:100F000084F48039910529F4E091B603F091B70398
:100F1000EACF803A9105F9F6E091B803F091B90370
:100F2000E2CF803D910509F0BBCEE091BE03F09188
:100F3000BF0308C0803C910509F0CFCEE091BC030F
:100F4000F091BD03309709F4C8CE6091EC03809115
:100F5000E9030995C2CE803F910509F0BECEE0912C
:100F6000C203F091C303309709F4B7CE6091ED034B
:100F700070E0762F66278091EC03682B613871054D
:100F800010F060E870E08EEE93E00995A6CE8A3FFF
:100F9000910509F081CFE091CE03F091CF0308C015
:100FA000883F910509F099CEE091CC03F091CD03F3
:100FB000309709F492CE099590CE833F9105A4F421
:100FC000E091C603F091C703309709F486CE809173
:100FD000ED038F77A0E88A9FC00111242091EC03D4
:100FE0002F77822B099579CE863F9105C9F6E0913E
:100FF000CA03F091CB03DCCF8C3F910529F4E0913B
:10100000D203F091D303D4CF8C3F91052CF4E0911F
:10101000D003F091D103CCCF8E3F910529F4E0911C
:10102000D403F091D503C4CF8F3F910509F055CE7D
:10103000E091D603F091D703BBCF8C2FDF91CF91F6
:101040001F910F91FF90EF900895CF93DF93E7E00A
:10105000F1E08491E3EFF0E0D491EFEDF0E0C491A2
:10106000CC2391F081110E949B02EC2FF0E0EE0F57
:10107000FF1FEE53FF4FA591B491EC91ED2381E05A
:1010800090E021F480E002C080E090E0DF91CF9119
:101090000895FF920F931F93CF93DF931F92CDB7C5
:1010A000DEB7182FF42E022F6F77422F82E6598376
:1010B0000E948C04612F6F77402F83E60E948C047E
:1010C0005981652F6F77402F86E00E948C046F2D29
:1010D0006F77402F86E20F90DF91CF911F910F9194
:1010E000FF900C948C049C018F7C8038910561F0FA
:1010F000203D310549F081E0203E310539F0203CAA
:10110000310521F080E0089581E008950895CF929F
:10111000DF92EF92FF920F931F93CF93DF931F9273
:10112000CDB7DEB7682F8EEB689F7001112409E5FB
:1011300012E0CC24C394D12CC6018E0D9F1D69836F
:101140000E94E503F80181938F01FFEFCF1ADF0AB8
:1011500069818FEBC816D10479F76093230580E08D
:1011600090E00F90DF91CF911F910F91FF90EF9042
:10117000DF90CF900C94C903862F653010F40C9447
:1011800087080895CF93DF93E82FF0E0E45AFE4FED
:10119000EF01CC54DF4FDF01A858BF4F8C918883FB
:1011A00084AD8C93808184AF80E480937C008091B7
:1011B0007A00806480937A0080917A0086FDFCCF6B
:1011C000809178002091790090E0922B23E0959512
:1011D00087952A95E1F78083DF91CF9108951F933A
:1011E000CF93DF93E82FF0E0E55EFE4F1081C12F33
:1011F000D0E0BE0183E0759567958A95E1F761704F
:1012000082E00E94C402BE0194E0759567959A95AC
:10121000E1F7617083E00E94C402BE0125E075958C
:1012200067952A95E1F7617084E00E94C402612FFE
:10123000617085E00E94C402BE017595679561707A
:1012400086E00E94C402D595C795D595C7956C2FA9
:10125000617087E00E94C4020E9493048BE891E0D1
:101260000197F1F7DF91CF911F9108954F925F920F
:101270006F927F928F929F92AF92BF92CF92DF92A6
:10128000EF92FF920F931F93CF93DF9300D000D084
:1012900000D0CDB7DEB7182F962E842EC82ED12CB5
:1012A000D601A45ABE4FCD0188589F4FFC018081C2
:1012B000DC96EC90DC97F12CE80EF11CCD018C54FF
:1012C0009F4FFC018081E80EF11C8C91E80EF11C0F
:1012D000F694E794F694E79421E030E040E050E0A3
:1012E00060E070E080E090E0012F0E948513A09103
:1012F0000E032A23A0910F033A23A09110034A233F
:10130000A09111035A23A09112036A23A091130301
:101310007A23B0911403A09115038B239A230E9482
:10132000A013A0E00E94BC1331F08FE790E09C0175
:101330002E193F097901C60181599B4F5C01DC01DF
:101340008C9190E0E816F90671F0DC968C91DC97B0
:1013500090E0E816F90639F0A858BF4F8C9190E05C
:10136000E816F90619F4992009F40DC1C601019691
:10137000FC01EE0FFF1F8E0F9F1FFC01E75AFD4F70
:1013800090818601000F111F97FFCDC0F801EC0D71
:10139000FD1DE75AFD4F9280911015C08110ADC020
:1013A000492F4F778FEF840F803120F481816E2D8C
:1013B0008F7706C04111A1C0409159026E2D8181E5
:1013C0000E948C049AC0811098C09F7797FE29C014
:1013D000618167FF26C0109159026F77412F82E625
:1013E0009E830E948C04692D6F77412F83E60E94B3
:1013F0008C0497019E81A92FB0E00E9470132FE703
:1014000030E040E050E00E941C13412F622F86E044
:101410000E948C048091160381116FC0412F60E0FF
:1014200040C0903408F041C080905902492E512CA0
:10143000519441945108052C000C66087708892FB7
:1014400090E0A0E0B0E09C01AD0124193509460907
:101450005709D7010E943B132FE730E040E050E0EE
:101460000E941C13420E531E641E751E0C0D1D1D82
:10147000F801E75AFD4F61816F77482D82E60E949F
:101480008C04692D6F77482D83E60E948C04482DCB
:1014900047FE09C061E086E00E948C0460E8640DAC
:1014A000482D86E28DCF642DFCCF953430F59134F4
:1014B00061F030F4903409F59701A4EAB0E008C077
:1014C000923449F1933459F118C09701A8ECB0E077
:1014D0000E9470132FE730E040E050E00E941C13A0
:1014E000BA01A9010C0D1D1DF801E75AFD4F20910D
:1014F00059026181892D0E944908F501E858FF4F82
:10150000D501DC968C91DC9780838C91DC968C9352
:10151000DC97EC9238C09701A0E4B6E0D9CF9701F0
:10152000A0EDB7E0D5CF2E2D0C0D1D1DF801E75A0B
:10153000FD4F828135E0E6E1F1E0DE011196019098
:101540000D923A95E1F787FF02C031E03B838F7738
:101550008C8330E0A92FB0E00E9470132FE730E0B9
:1015600040E050E00E941C132D8320E0AE014F5F4D
:101570005F4F65E070E088ED93E00E94780341E002
:1015800060E08FE71DCF26960FB6F894DEBF0FBE42
:10159000CDBFDF91CF911F910F91FF90EF90DF9022
:1015A000CF90BF90AF909F908F907F906F905F9003
:1015B0004F9008958F929F92BF92CF92DF92EF92B9
:1015C000FF920F931F93CF93DF931F92CDB7DEB798
:1015D000DC0111968C911197803309F0FFC11296AE
:1015E000EC9112974E2F50E0FA013197E331F1055B
:1015F00008F0F4C14D01EC5BFF4F0C947F13139680
:101600008C9113978C3308F0E9C190E014962C91DB
:101610001497FC01EE0FFF1FE80FF91FE75AFD4F6B
:10162000218312820196FC01EE0FFF1F8E0F9F1F78
:10163000FC01E75AFD4F80E81DC0FD0183818C331A
:1016400008F0CCC190E02481FC01EE0FFF1FE80FF1
:10165000F91FE75AFD4F218312820196FC01EE0F1C
:10166000FF1F8E0F9F1FFC01E75AFD4F15968C91AF
:1016700015978068808313968C910F90DF91CF919E
:101680001F910F91FF90EF90DF90CF90BF909F90B0
:101690008F900C945C04FD0183818C3308F09EC113
:1016A00090E0FC01EE0FFF1FE80FF91FE75AFD4F16
:1016B000118212820196FC01EE0FFF1F8E0F9F1FF9
:1016C000FC01E75AFD4F81E9808388C113968C9114
:1016D00013978C3308F082C116962C91169790E0E0
:1016E00014963C911497FC01EE0FFF1FE80FF91FB1
:1016F000E75AFD4F318315963C913068328301964D
:10170000FC01EE0FFF1F8E0F9F1FFC01E75AFD4FDC
:10171000822F203408F08FE380588083F401838186
:10172000ACCF13968C9113978C3308F057C190E08F
:10173000FC01EE0FFF1FE80FF91FE75AFD4F14964B
:101740002C9114972068218315962C911597206869
:1017500022830196FC01EE0FFF1F8E0F9F1FFC01DD
:10176000E75AFD4F16968C911697805883CFFD014E
:1017700083818C3308F032C1368190E02481DC0112
:10178000AA0FBB1FA80FB91FA75ABD4F11962C93C4
:1017900011972581206812962C93EFEFE30FE43028
:1017A00028F4F0E0E95AFE4F208101C029E40196B7
:1017B000FC01EE0FFF1F8E0F9F1FFC01E75AFD4F2C
:1017C00020582083D40157CFFD0183818C3308F04A
:1017D00005C190E0FC01EE0FFF1FE80FF91FE75A6B
:1017E000FD4F118214962C91B0E82B9F900111248B
:1017F000D40115963C911597232B228316962C9194
:1018000016970196FC01EE0FFF1F8E0F9F1FFC0124
:10181000E75AFD4F20832FCFFD0103810C3308F0E1
:10182000DDC08481811102C0802F27CF21E030E00C
:1018300040E050E060E070E080E090E00E948513BE
:10184000E0910E032E2BE0910F033E2BE09110034D
:101850004E2BE09111035E2BE09112036E2BE09171
:1018600013037E2BE09114038E2BE09115039E2B26
:1018700020930E0330930F034093100350931103F2
:1018800060931203709313038093140390931503D2
:10189000A5C013968C91882321F081E080931603D4
:1018A00002C010921603F4019381953008F096C09F
:1018B000FEEB9F9F9001112409E512E0C9018955B3
:1018C00092406C01D8016D918D017601EA0EFB1EEC
:1018D000C70169830E9406136981681719F0C7015F
:1018E0000E940E13B3E007311B0761F761E082E14C
:1018F0000E94C40268EE73E080E090E00E94F4026F
:1019000060E082E10E94C4026AEF70E080E090E053
:101910000E94F40261E082E10E94C4026AEF70E07A
:1019200080E090E00E94F40260E082E10F90DF919D
:10193000CF911F910F91FF90EF90DF90CF90BF90CC
:101940009F908F900C94C402FD018381853008F034
:1019500045C00F90DF91CF911F910F91FF90EF90B5
:10196000DF90CF90BF909F908F900C94870810E0ED
:1019700040E061E0812F0E9436091F5F1C33C1F7F0
:101980002DC013968C919FEF980F903138F580936E
:10199000590224C0FD0183818F3700F59481981787
:1019A000E8F0082F10E08FE7C82ED12CE12CF12CA5
:1019B000D40114968C9190E0801791077CF0B09040
:1019C00059020E94F812A70196010E941C134B2D88
:1019D000802F0E948C040F5F1F4FEACF0F90DF9182
:1019E000CF911F910F91FF90EF90DF90CF90BF901C
:1019F0009F908F900895DC01ED91FC910190F08112
:101A0000E02D0994CF93DF93CDB7DEB7CE5BD1093C
:101A10000FB6F894DEBF0FBECDBF789484B5826058
:101A200084BD84B5816084BD85B5826085BD85B582
:101A3000816085BD80916E00816080936E00109200
:101A4000810080918100826080938100809181007B
:101A5000816080938100809180008160809380000C
:101A60008091B10084608093B1008091B00081606A
:101A70008093B00080917A00846080937A00809196
:101A80007A00826080937A0080917A0081608093EE
:101A90007A0080917A00806880937A001092C10069
:101AA00061E081E00E94B90161E081E00E94C4022E
:101AB00061E082E00E94B90161E083E00E94B90127
:101AC00061E084E00E94B90161E085E00E94B90113
:101AD00061E086E00E94B90161E087E00E94B901FF
:101AE00061E082E10E94B90162E083E10E94B901F4
:101AF0000E942508892B71F560E082E10E94C402F2
:101B00000E941A02683873418105910528F40E94E9
:101B10002508892BA9F31EC061E082E10E94C4025E
:101B200064E170E080E090E00E94F40260E082E115
:101B30000E94C40200E010E060E0C8010E940E13A1
:101B40000F5F1F4F011534E01307B1F761E082E129
:101B50000E94C4028DEF93E00E94E503082F8EEFF0
:101B600093E00E94E503182F8FEF93E00E94E503B6
:101B70000B3A29F41D3319F4863609F4C5C215E071
:101B800061E082E10E94C4026CE271E080E090E0DA
:101B90000E94F40260E082E10E94C4026CE271E003
:101BA00080E090E00E94F402115051F760E080E084
:101BB00090E00E94C90381E0898384E58A831B82C7
:101BC00080E88C8393E59D831E828F8393E39887BF
:101BD00019868A879BE49B871C868D8797E49E875E
:101BE0001F86888B97E6998B1A8A8B8B9DE69C8B38
:101BF0001D8A8E8B99E59F8B188E898F93EB9A8F18
:101C00008B8F9BE89C8F2AE72D8F1E8E8F8F26E56A
:101C100028A319A28AA325E52BA31CA28DA325E343
:101C20002EA31FA288A72CE429A71AA68BA727E218
:101C30002CA71DA68EA72DE22FA718AA89AB2EE6EA
:101C40002AAB1BAA8CAB2AE52DAB1EAA8FAB24EBCB
:101C500028AF89AF9AAF2BE72BAF1CAE8DAF2DE02D
:101C60002EAF1FAE21968FAF219727E522962FAF7B
:101C7000229723961FAE239724968FAF249727E3AE
:101C800025962FAF259726961FAE269727968FAFBE
:101C900027972DE428962FAF289729961FAE2997CE
:101CA0002A968FAF2A9728E22B962FAF2B972C9648
:101CB0001FAE2C972D968FAF2D972EE22E962FAF1D
:101CC0002E972F961FAE2F9760968FAF60972FE6B7
:101CD00061962FAF619762961FAE629763968FAF42
:101CE00063972BE564962FAF649765961FAE659753
:101CF00066968FAF669725EB67962FAF67976896C6
:101D00008FAF689769969FAF69972CE76A962FAF58
:101D10006A976B961FAE6B976C968FAF6C972FE0A0
:101D20006D962FAF6D976E961FAE6E976F968FAFB5
:101D30006F972DE1A0962FAFA097A1961FAEA19708
:101D4000A2968FAFA29729E3A3962FAFA397A4964D
:101D50001FAEA497A5968FAFA5972EE4A6962FAF9A
:101D6000A697A7961FAEA797A8968FAFA89729E228
:101D7000A9962FAFA997AA961FAEAA97AB968FAF39
:101D8000AB972FE2AC962FAFAC97AD961FAEAD9749
:101D9000AE968FAFAE9720E7AF962FAFAF97E09696
:101DA0001FAEE097E1968FAFE1972CE5E2962FAF5B
:101DB000E297E3961FAEE397E4968FAFE49726EBA6
:101DC000E5962FAFE597E6968FAFE697E7969FAF3C
:101DD000E7972DE7E8962FAFE897E9961FAEE997CA
:101DE000EA968FAFEA9721E1EB962FAFEB97EC964F
:101DF0001FAEEC97ED968FAFED972AE3EE962FAFDF
:101E0000EE97EF961FAEEF97C158DF4F8883CF57FD
:101E1000D0402BE3C058DF4F2883C058D040CF5765
:101E2000DF4F1882C158D040CE57DF4F8883C25849
:101E3000D04023E4CD57DF4F2883C358D040CC5740
:101E4000DF4F1882C458D040CB57DF4F8883C55826
:101E5000D0402AE2CA57DF4F2883C658D040C9571E
:101E6000DF4F1882C758D040C857DF4F8883C85803
:101E7000D04020E3C757DF4F2883C958D040C6570A
:101E8000DF4F1882CA58D040C557DF4F8883CB58E0
:101E9000D04021E7C457DF4F2883CC58D040C357E8
:101EA000DF4F1882CD58D040C257DF4F8883CE58BD
:101EB000D0402DE5C157DF4F2883CF58D040C057C1
:101EC000DF4F1882C059D040CF56DF4F8883C159A9
:101ED000D04027EBCE56DF4F2883C259D040CD5695
:101EE000DF4F8883C359D040CC56DF4F9883C45905
:101EF000D0402EE7CB56DF4F2883C559D040CA5675
:101F0000DF4F1882C659D040C956DF4F8883C75962
:101F1000D04023E1C856DF4F2883C859D040C75668
:101F2000DF4F1882C959D040C656DF4F8883CA593F
:101F3000D0402DE3C556DF4F2883CB59D040C4563F
:101F4000DF4F1882CC59D040C356DF4F8883CD591C
:101F5000D0402EE3C256DF4F2883CE59D040C15621
:101F6000DF4F1882CF59D040C056DF4F8883C05A08
:101F7000D04024E4CF55DF4F2883C15AD040CE55FE
:101F8000DF4F1882C25AD040CD55DF4F8883C35AE5
:101F9000D0402BE2CC55DF4F2883C45AD040CB55DC
:101FA000DF4F1882C55AD040CA55DF4F8883C65AC2
:101FB000D04021E3C955DF4F2883C75AD040C855C8
:101FC000DF4F1882C85AD040C755DF4F8883C95A9F
:101FD000D04022E7C655DF4F2883CA5AD040C555A6
:101FE000DF4F1882CB5AD040C455DF4F8883CC5A7C
:101FF000D0402EE5C355DF4F2883CD5AD040C2557F
:10200000DF4F1882CE5AD040C155DF4F8883CF5A58
:10201000D04028EBC055DF4F2883C05BD040CF5461
:10202000DF4F8883C15BD040CE54DF4F9883C25BC3
:10203000D0409FE7CD54DF4F9883C35BD040CC5452
:10204000DF4F1882C45BD040CB54DF4F8883C55B21
:10205000D040CA54DF4F1882C65BD040C954DF4F0E
:102060001882C75BD040C854DF4F1882C85BD0408D
:10207000C754DF4F1882C95BD040C654DF4F188267
:10208000CA5BD040C554DF4F1882CB5BD040C454EC
:10209000DF4F1882CC5BD040C354DF4F1882CD5B3A
:1020A000D040C254DF4F1882CE5BD04000E010E039
:1020B000AE014F5F5F4F6A014E015FEB850E911CD1
:1020C00076015801AC18BD08D7016D917D01CD0195
:1020D0008A0D9B1D0E94C903E814F904A9F7025454
:1020E0001F4F083FB2E01B0759F76BEA8DEF93E0F3
:1020F0000E94C9036DE38EEF93E00E94C90366E678
:102100008FEF93E00E94C90380E090E00E94E50316
:102110000E9487080E941A0260935502709356022B
:1021200080935702909358022AE0E22EF12C10E09F
:10213000812F0E94EF08812F0E94C20841E060E0D9
:10214000812F0E9436091F5F1C3391F7E1E0EE1AE0
:10215000F10869F78AED9AE09093C3038093C20374
:102160008CEB98E09093BD038093BC0383E0809355
:10217000E803E091D803F091D903A089B18982E006
:102180008C93A485B5851C92A685B7858FE38C9327
:10219000108EA489B58986E08C93A289B3898C912D
:1021A00080618C93A289B3898C9188608C93A28979
:1021B000B3898C9180688C930288F389E02D8081AB
:1021C0008F7D808381E08093DA031092DC0310928C
:1021D000DB031092E3031092E2031092E1031092EA
:1021E000E0038FEF9FEF9093E5038093E4039093D8
:1021F000E7038093E60310926E041092EB031092B3
:10220000EA031092E9031092EC031092ED0380911F
:10221000E8038170826081608093E8038091D80335
:102220009091D903DC01ED91FC910190F081E02DBA
:102230006EEF099561E082E10E94C40210E00E9405
:102240009304812F0E94EF080E949304812F0E9423
:10225000C2080E94930440E060E0812F0E9436098A
:102260001F5F1C3361F70E942508892B09F0DFC02E
:102270001092E8030E941A02C0905502D0905602B4
:10228000E0905702F09058026C157D058E059F0571
:10229000B1F00E941A02DC01CB018C199D09AE0934
:1022A000BF0985369105A105B10508F441C00E941A
:1022B0001A026C157D058E059F0561F419C00E94F8
:1022C0001A02A7019601261B370B480B590BDA019E
:1022D000C901E7CF0E941A02DC01CB018C199D09CC
:1022E000AE09BF098E359140A105B10570F020C03F
:1022F0000E941A02C61AD70AE80AF90A4EE5C4165D
:1023000041E0D406E104F10498F460E082E10E9427
:10231000C40210E040E061E0812F0E9436091F5F97
:102320001C33C1F764EF71E080E090E00E94F4029A
:1023300020E040E050E060E070E088ED93E00E9433
:1023400078030E941A02609355027093560280939C
:102350005702909358020E942508892B09F067C004
:1023600010E00E949304812F0E94EF080E949304C2
:10237000812F0E94C2081F5F1C3399F78CE5C82E7D
:1023800081E0D82E98E9E92E91E0F92E11E0D601EE
:102390008D916D01F70121917F0190E0821B9109E0
:1023A00097FF03C0919581959109039784F010934D
:1023B000590260E082E10E94C40264E670E080E0BD
:1023C00090E00E94F40261E082E10E94C4021F5F7B
:1023D0001131E9F600E010E0F801E45AFE4F82A95D
:1023E00090E0E259FF4F2081821B910997FF03C0C3
:1023F00091958195910903978CF0802F0E94870811
:1024000060E082E10E94C4026AEF70E080E090E048
:102410000E94F40261E082E10E94C4020F5F1F4F3C
:1024200005301105C9F683E08093E80394CF0E943C
:10243000AF0100CFCF93DF93A7E1B3E013961C92D7
:102440001E92129748EE53E060E070E014964D93B0
:102450005D936D937C93179788E091E011969C9320
:102460008E9385EC90E01D969C938E931C9784EC44
:1024700090E01F969C938E931E9780EC90E051966F
:102480009C938E93509781EC90E053969C938E93FF
:10249000529782EC90E055969C938E93549786ECDD
:1024A00090E057969C938E93569759961C92599705
:1024B0005A961C925A975B961C925B975C961C925C
:1024C0005C97E4EBF3E0B5A3A4A316A217A210A6B1
:1024D00015A614A617A616A68FEF9FEF91AB80AB9B
:1024E00093AB82AB83E08093E80315AA17AA16AAE0
:1024F00010AE11AE10926E0480E8AEEEB3E0ED01C6
:1025000019928A95E9F7118210821382128215823C
:1025100014821782168211861086138612861586FB
:10252000148617861686118A108A138A128A158ACB
:10253000148A178A168A118E108E138E128E158E9B
:10254000148E178E168E11A210A213A212A2DF9162
:10255000CF9108958F929F92AF92BF92CF92DF92C8
:10256000EF92FF92CF93DF93EC01688179818A81AA
:102570009B81611571058105910521F464E279ED76
:102580008BE597E02DE133EF41E050E00E941C1312
:1025900049015A019B01AC01A7EAB1E40E943B1337
:1025A0006B017C01ACEEB4EFA50194010E944913CC
:1025B000DC01CB018C0D9D1DAE1DBF1DB7FF03C0FF
:1025C0000197A109B04888839983AA83BB83BC0182
:1025D000CD019F77DF91CF91FF90EF90DF90CF906B
:1025E000BF90AF909F908F9008950E94AA12089577
:1025F00080E091E00E94AA12089560930001709318
:10260000010180930201909303010895F999FECF8F
:1026100092BD81BDF89A992780B50895262FF99922
:10262000FECF1FBA92BD81BD20BD0FB6F894FA9AB5
:10263000F99A0FBE01960895052E97FB1EF400949B
:102640000E94331357FD07D00E944E1307FC03D09E
:102650004EF40C94331350954095309521953F4F8F
:102660004F4F5F4F089590958095709561957F4F7E
:102670008F4F9F4F08950E947013A59F900DB49F98
:10268000900DA49F800D911D11240895B7FF0C9407
:102690003B130E943B13821B930B0895A1E21A2E59
:1026A000AA1BBB1BFD010DC0AA1FBB1FEE1FFF1FF6
:1026B000A217B307E407F50720F0A21BB30BE40B46
:1026C000F50B661F771F881F991F1A9469F760958D
:1026D0007095809590959B01AC01BD01CF01089547
:1026E000A29FB001B39FC001A39F700D811D112453
:1026F000911DB29F700D811D1124911D0895EE0F43
:10270000FF1F0590F491E02D09940F93083090F08D
:10271000982F872F762F652F542F432F322F222764
:102720000850F4CF220F331F441F551F661F771F19
:10273000881F991F0A95B2F70F91089597FB10F81B
:10274000169400080F93083098F00850232F342F68
:10275000452F562F672F782F892F902DF4CF059472
:1027600097958795779567955795479537952795C9
:102770000A95AAF70F9108950024A7FD00942A173F
:1027800030054005500560057005800590050895E9
:0E27900081E090E0F8940C94CD13F894FFCF04
:10279E0001000000000000004601AF00DE008D01C8
:1027AE000F01ED00010143100000002A3A1008004D
:1027BE0018283830203222130B031B2B3B332311E6
:1027CE0009150D051D2D3D35250119170F071F2F55
:1027DE003F37272939160E061E2E3E362631211476
:0C27EE000C041C2C3C34244041424300ED
:00000001FF
